:020000040000FA
:0600000084EF09F012007C
:0608000084EF09F0120074
:020808001200DC
:020818001200CC
:02082A000000CC
:04082C00040118515A
:10083000600BE842E842E842E842E842000901E091
:1008400055D01951070A51E00B0A4FE0070A40E062
:10085000010A2CE00B0A28E0020A26E0030A22E043
:10086000080A12E0010A0EE00F0A0AE0030A01E09A
:100870003CD00001010E616F0001040E846F36D080
:1008800036D834D090D832D00001010E616F00010B
:10089000860E626F000E636F000185930001010EEA
:1008A000666F24D0A6D822D0F2D820D00001010E45
:1008B000616F04011C510001626F636B870E622738
:1008C000000E6323000185930001010E666F0ED0B8
:1008D0000001010E616F04011C51EA6A870FE96E85
:1008E000000EEA221AC4EFFF01D000D01200800EE1
:1008F0000401185D57E11B51030A34E0010A10E0BE
:10090000030A01E04DD00001010E616F00013E0EAF
:10091000626F120E636F120E0001666F676B40D03C
:100920000001010E616F04011A51F66EF76AD8904A
:10093000F636F7369E0EF626120EF7220900F5CF90
:1009400062F00A00F5CF63F0020E0001F76A62253B
:10095000F66E6351F7220900F5CF66F00A00F5CF75
:1009600067F01ED00001010E616F04011A51F66E8E
:10097000F76AD890F636F736A20EF626120EF72250
:100980000900F5CF62F00A00F5CF63F062C0F6FF10
:1009900063C0F7FF0800F5500001666F676B00D079
:1009A0000001858312000001010E616F00010F0E2E
:1009B000836F0001710E816F0F0E826F5BEC08F088
:1009C0000001010E836F0001870E816F000E826FA0
:1009D0005BEC08F01AC486F004011A5104E100012E
:1009E000050E846F05D00001060E846F67EC08F0D9
:1009F00012000401206B216B040118511F0B020A25
:100A000014E0030A0EE0010A01E033D00001010EF8
:100A1000616F04012081000185A102D004012083BF
:100A200028D00001010E616F24D00001010E616F1A
:100A300004011C510F0B080DF350036A000F026EE6
:100A4000040E03221C51800B01E0010E040DF35033
:100A500000010224646F000E0320656F64C0E9FF8B
:100A600065C0EAFFEF50040B03E00401010E206FA4
:100A700000D0000161050AE10001200E626F040E42
:100A8000636F000185930001020E666F120004017E
:100A90001A0510E118511F0B00090CE10001010EAD
:100AA000616F030E0401195D03E10001858102D02D
:100AB0000001859104011A513AE118511F0B0208F7
:100AC00036E11C510F0B000932E00001010E616F8D
:100AD00004011C510F0B080DF350036A000F026E46
:100AE000040E03221C51800B01E0010E040DF35093
:100AF00000010224646F000E0320656F030E0401E1
:100B0000195D07E1840E64C0E9FF65C0EAFFEF6E7E
:100B10000ED01CAF06D064C0E9FF65C0EAFFEF6AE3
:100B200006D0880E64C0E9FF65C0EAFFEF6E1200D0
:100B30006C5002E0000E01D0010E00090BE0040130
:100B400000513C0BE842E8420D0802E10CD801D00C
:100B500013D808D06C5002E0000E01D0010E040939
:100B600001E01AD812000001606B616B666B676B65
:100B700016EC04F064EF06F0020E0001605D0AE17D
:100B80007CD8040100BD03D0C80E006F02D0880ECF
:100B9000006F01D0DFD81200040E0001845D0AE16D
:100BA0001AC46EFF6E50000803E2050E846F02D077
:100BB000030E846F000160050AE10BD8040104BD37
:100BC00003D0C80E046F02D0880E046F01D0C2D8C3
:100BD00012000001080E665D000E675905E266C04E
:100BE00069F067C06AF003D0080E696F6A6B040190
:100BF0000493049100016A510401041369C005F4CF
:100C000000016951665D666F6A516759676F200E12
:100C1000646F040E656F000185A318D0000169514F
:100C20006A1113E062C0F6FF63C0F7FF0800F550D9
:100C300064C0E9FF65C0EAFFEF6E642B000E652318
:100C4000622B632369076A5BE9D716D000016951FB
:100C50006A1112E062C0E9FF63C0EAFFEF5064C0AE
:100C6000E9FF65C0EAFFEF6E642B000E6523622B7F
:100C7000632369076A5BEAD71200030E04010015BB
:100C800000016C6F01C46BF066516B25666F675194
:100C90006C21676F200E626F040E636F6B516C11D5
:100CA00012E062C0E9FF63C0EAFFEF5064C0E9FFF1
:100CB00065C0EAFFEF6E642B000E6523622B632391
:100CC0006B076C5BEBD71200000161510CE1040172
:100CD000080E016F180E026F040E036F840E006F72
:100CE0000401046F35D0040118AF22D00001665111
:100CF00004011E5D0001675104011F5904E21EC476
:100D000066F01FC467F065DF0001010E606F04012B
:100D1000080E016F180E026F040E036F800E006F35
:100D20000401200E066F040E076FC80E046F10D06A
:100D30000001020E606F0401056BC80E046F040110
:100D4000080E016F200E026F040E036FC80E006FB5
:100D50006D9812000001606B0401080E016F180EFF
:100D6000026F040E036F880E006F0401046B120003
:100D7000800EF16E926A896A936A8A6A946A8B6AB3
:100D80000101010E5C6F12008B6A946A200E8916B5
:100D90009216F16A0101416B426B496B516B526BC8
:100DA000010E4A6F4B6B4C6B436B446B4F6B506B3C
:100DB000556B566B576B5A6F5B6B5C6B970ED56EB2
:100DC000F50ECD6ED5DF89868B8E898A120000C222
:100DD000E6FF6DEC09F0E5521200060E0001845D9D
:100DE00003E36D50020B01E015D015D89EA012D080
:100DF0009E90CF6ACE6A0101552B555103080AE235
:100E0000B0D801015651000804E25607020E556F92
:100E100001D0556B12000001400E7E6F0001010EE3
:100E20007C6F010E7D6FA2EC08F0000901E188D013
:100E30000101006B01010151520A5BE0030A2CE041
:100E4000010A22E0AF0A1EE0C40A15E0790A0CE0AC
:100E5000420A01E065D00101036B01010D0E046F30
:100E60000101040E006F5DD00101030E026F01014C
:100E7000020E006F56D00101140E566F0101010ED3
:100E8000006F4FD0FF004DD073DF89868B8E898A2B
:100E90000101010E006F45D00101010E006F01013B
:100EA000025102E1899A89960101020502E1898ACB
:100EB0008996020E0101025D02E1899A8986030E7C
:100EC0000101025D02E1898A898603C18AFF010E60
:100ED0000201006F016B7BDF8B9E010E0201006F30
:100EE000016B75DF8B8E010E0201006F016B6FDFEE
:100EF00018D00101010E006F8B9E89880101020547
:100F000002E18B8E89888996020E0101025D01E162
:100F10008986899A030E0101025D01E1898A01D067
:100F200000D0010100510CE004010CBF09D000C148
:100F30007AF00001010E786F010E796F7CEC08F0F9
:100F40001200F294D76AD66AD76AF29401014F6B05
:100F5000506B4D6B4E6B526B52C151F1010E4A6F8B
:0E0F6000120089A802D0899801D08988120059
:020F6E006DA66E
:100F70000FD802D06DB613D80001840508E16DBA10
:100F800006D0686A696A69806988020E846F1200F7
:100F90006D6A696A6D860001010E846F12006D6AC8
:100FA000696A0001846B1200CFEF07F000018451E1
:100FB00001E13AD06850040B04E06950040B01E0F1
:100FC00038D86DB231D06850010B04E06950010B84
:100FD00001E050D86850100B04E06950100B01E09C
:100FE00024D86850400B04E06950400B01E037D82A
:100FF0006850200B04E06950200B01E032D86850A3
:10100000020B04E06950020B01E032D8030E00012C
:10101000845D01E209D06850080B06E06950080BB6
:1010200003E098EC05F068961200698468986D8278
:1010300012006D92699468941200000185A10ED08F
:10104000F8DF6D840001080E7F6F070E806F7F0749
:10105000000E805B7F518011FAE16D941200689C54
:10106000120070A003D0AAEC06F07090689A1200EB
:10107000689212006A6A686A9F0E6B6E7B0E696ED8
:101080006E6A00010F0E836F0001710E816F0F0EEB
:10109000826F11D8160E706E68A602D06896FCD7C3
:1010A0006D98AAEC06F0000185910001866B0001A5
:1010B000030E846F120081C0E9FF82C0EAFF0001C5
:0E10C000835104E0EE6A00018307F9D71200A5
:0210CE0000011F
:1010D000776B1E0E716E0401400E096F280E0A6FA9
:1010E000040E0B6F880E086F0401680E0E6F040E5D
:1010F0000F6F400E0C6F120000017A51400802E29F
:10110000400E7A6F7B6B7A517B5D13E27B51EA6A0A
:101110007825E96E7951EA22EF50E66E7B51EA6A52
:10112000680FE96E040EEA22E552E750EF6E7B2B62
:10113000EAD77AC00DF4400E04010C170C7D880E1E
:101140000C1312000001776B040108BF25D0095170
:101150000001D8807E5502E209C47EF0776B7E5193
:10116000775D13E27751EA6A280FE96E040EEA22EE
:10117000EF50E66E7751EA6A7C25E96E7D51EA22EE
:10118000E552E750EF6E772BEAD70401400E096F66
:101190000817087D880E08130001775100D012004F
:1011A0002A0EF66E080EF76E000EF86E00010900AA
:1011B000F550726F0900F550736F03E1726701D04B
:1011C0003DD00900F5506D6F0900F5506E6F0900B4
:1011D000F5506F6F09000900F550E96E0900F550F0
:1011E000EA6E090009000900F550706F0900F5501A
:1011F000716F09000900F6CF74F0F7CF75F0F8CFE2
:1012000076F06DC0F6FF6EC0F7FF6FC0F8FF00010B
:10121000705302E1715307E00900F550EE6E70075C
:10122000F8E27107F9D774C0F6FF75C0F7FF76C012
:0E123000F8FF00017207000E735BBFD71200BB
:02123E0012019B
:10124000000200000008D804010F000001020002A3
:1012500009022000010100803209040000020000A0
:10126000000007050103400020070581034000201E
:1012700004030904100343006F0063006B00700057
:10128000690074001A03540061006E006B006E0068
:10129000650074007A007400650069006C005012EB
:0812A000501270127412841246
:0812A80005D810D8EDEC06F0AA
:1012B000FCD712000F0EC112140E6F6E0001846B6A
:1012C0000001856B0001866BC4EF06F0B7EC07F0F8
:0A12D0006FBE02D0D6EC07F012004A
:0612DA00FF0EE350056E5B
:1012E000EF0E01D0F30EE76EE72E74EF09F00C0E4F
:1012F000046EE76AE72E7AEF09F0042E79EF09F021
:08130000052E72EF09F0120046
:0813080013EE00F023EE00F0EB
:10131000F86A019CD0EC08F092EC09F054EC09F06A
:04132000FBD71200E5
:021324001200B5
:00000001FF
